:020000040800F2
:1000000000C00020293D00080D3D00080F3D0008FC
:10001000113D0008133D0008153D000800000000D8
:10002000000000000000000000000000173D000874
:10003000193D0008000000001B3D00081D3D0008A0
:10004000713D0008713D0008713D0008713D0008D8
:10005000713D0008713D0008713D0008713D0008C8
:10006000713D0008713D0008713D000839350008F8
:10007000713D0008713D0008713D0008713D0008A8
:10008000713D0008713D0008713D0008713D000898
:10009000713D0008713D0008713D0008713D000888
:1000A000713D0008713D0008713D0008713D000878
:1000B000713D0008713D0008713D0008713D000868
:1000C000713D0008713D0008713D0008713D000858
:1000D000713D0008713D0008713D0008713D000848
:1000E000713D0008713D0008713D0008713D000838
:1000F000713D0008713D0008713D0008713D000828
:10010000713D0008713D0008713D0008713D000817
:10011000713D0008713D0008713D0008713D000807
:10012000713D0008713D0008713D0008713D0008F7
:1001300000000000000000000000000000000000BF
:1001400000000000000000000000000000000000AF
:10015000000000000000000000000000000000009F
:10016000000000000000000000000000000000008F
:10017000000000000000000000000000000000007F
:10018000000000000000000000000000000000006F
:10019000000000000000000000000000000000005F
:1001A000000000000000000000000000000000004F
:1001B000000000000000000000000000000000003F
:1001C000000000000000000000000000000000002F
:1001D000000000000000000000000000000000001F
:0401E0005FF8E0F1F3
:1001E80010B5054C237833B9044B13B10448AFF369
:1001F80000800123237010BD8C0000200000000047
:100208000846000808B5034B1BB103490348AFF380
:10021800008008BD0000000090000020084600088B
:10022800034613F8012B002AFBD1181A013870472E
:1002380081F0004102E000BF83F0004330B54FEA8F
:1002480041044FEA430594EA050F08BF90EA020FFC
:100258001FBF54EA000C55EA020C7FEA645C7FEA8F
:10026800655C00F0E2804FEA5454D4EB5555B8BFB2
:100278006D420CDD2C4480EA020281EA030382EA23
:10028800000083EA010180EA020281EA0303362DB5
:1002980088BF30BD11F0004F4FEA01314FF4801C88
:1002A8004CEA113102D0404261EB410113F0004F9A
:1002B8004FEA03334CEA133302D0524263EB430351
:1002C80094EA050F00F0A780A4F10104D5F1200EEF
:1002D8000DDB02FA0EFC22FA05F2801841F100014A
:1002E80003FA0EF2801843FA05F359410EE0A5F11E
:1002F80020050EF1200E012A03FA0EFC28BF4CF04F
:10030800020C43FA05F3C01851EBE37101F0004504
:1003180007D54FF0000EDCF1000C7EEB00006EEB11
:100328000101B1F5801F1BD3B1F5001F0CD349089B
:100338005FEA30004FEA3C0C04F101044FEA4452F2
:1003480012F5800F80F09A80BCF1004F08BF5FEA79
:10035800500C50F1000041EB045141EA050130BD59
:100368005FEA4C0C404141EB010111F4801FA4F1FC
:100378000104E9D191F0000F04BF01460020B1FA51
:1003880081F308BF2033A3F10B03B3F120020CDA89
:100398000C3208DD02F1140CC2F10C0201FA0CF067
:1003A80021FA02F10CE002F11402D8BFC2F1200CCC
:1003B80001FA02F120FA0CFCDCBF41EA0C01904082
:1003C800E41AA2BF01EB0451294330BD6FEA0404CB
:1003D8001F3C1CDA0C340EDC04F11404C4F12002B6
:1003E80020FA04F001FA02F340EA030021FA04F3C8
:1003F80045EA030130BDC4F10C04C4F1200220FA1F
:1004080002F001FA04F340EA0300294630BD21FA5C
:1004180004F0294630BD94F0000F83F4801306BF22
:1004280081F480110134013D4EE77FEA645C18BF16
:100438007FEA655C29D094EA050F08BF90EA020FAD
:1004480005D054EA000C04BF1946104630BD91EAA5
:10045800030F1EBF0021002030BD5FEA545C05D1A8
:100468004000494128BF41F0004130BD14F58004E7
:100478003CBF01F5801130BD01F0004545F0FE415B
:1004880041F470014FF0000030BD7FEA645C1ABF90
:10049800194610467FEA655C1CBF0B46024650EAC7
:1004A800013406BF52EA033591EA030F41F40021F3
:1004B80030BD00BF90F0000F04BF0021704730B579
:1004C8004FF4806404F132044FF000054FF000014E
:1004D80050E700BF90F0000F04BF0021704730B50F
:1004E8004FF4806404F1320410F0004548BF4042E4
:1004F8004FF000013EE700BF42004FEAE2014FEA39
:1005080031014FEA02701FBF12F07F4393F07F4F13
:1005180081F06051704732F07F4208BF704793F016
:100528007F4F04BF41F40021704730B54FF4607429
:1005380001F0004521F000411CE700BF50EA01022C
:1005480008BF704730B54FF000050AE050EA0102D5
:1005580008BF704730B511F0004502D5404261EB45
:1005680041014FF4806404F132045FEA915C3FF486
:10057800D8AE4FF003025FEADC0C18BF03325FEA23
:10058800DC0C18BF033202EBDC02C2F1200300FAD4
:1005980003FC20FA02F001FA03FE40EA0E0021FAF9
:1005A80002F11444BDE600BF70B54FF0FF0C4CF4E7
:1005B800E06C1CEA11541DBF1CEA135594EA0C0F99
:1005C80095EA0C0F00F0DEF82C4481EA030621EAD4
:1005D8004C5123EA4C5350EA013518BF52EA03350F
:1005E80041F4801143F4801338D0A0FB02CE4FF0C1
:1005F8000005E1FB02E506F00042E0FB03E54FF0F1
:100608000006E1FB03569CF0000F18BF4EF0010EE8
:10061800A4F1FF04B6F5007F64F5407404D25FEAE4
:100628004E0E6D4146EB060642EAC62141EA555197
:100638004FEAC52040EA5E504FEACE2EB4F1FD0CD9
:1006480088BFBCF5E06F1ED8BEF1004F08BF5FEA57
:10065800500E50F1000041EB045170BD06F0004609
:1006680046EA010140EA020081EA0301B4EB5C04B6
:10067800C2BFD4EB0C0541EA045170BD41F48011AE
:100688004FF0000E013C00F3AB8014F1360FDEBFD3
:10069800002001F0004170BDC4F10004203C35DAAF
:1006A8000C341BDC04F11404C4F1200500FA05F332
:1006B80020FA04F001FA05F240EA020001F00042D3
:1006C80021F0004110EBD37021FA04F642EB060149
:1006D8005EEA430E08BF20EAD37070BDC4F10C0473
:1006E800C4F1200500FA04F320FA05F001FA04F237
:1006F80040EA020001F0004110EBD37041F1000123
:100708005EEA430E08BF20EAD37070BDC4F120052D
:1007180000FA05F24EEA020E20FA04F301FA05F295
:1007280043EA020321FA04F001F0004121FA04F23D
:1007380020EA020000EBD3705EEA430E08BF20EA0D
:10074800D37070BD94F0000F0FD101F00046400047
:1007580041EB010111F4801F08BF013CF7D041EAC9
:10076800060195F0000F18BF704703F000465200CD
:1007780043EB030313F4801F08BF013DF7D043EA9E
:100788000603704794EA0C0F0CEA135518BF95EA54
:100798000C0F0CD050EA410618BF52EA4306D1D1DB
:1007A80081EA030101F000414FF0000070BD50EAFA
:1007B800410606BF1046194652EA430619D094EA84
:1007C8000C0F02D150EA013613D195EA0C0F05D16E
:1007D80052EA03361CBF104619460AD181EA0301C2
:1007E80001F0004141F0FE4141F470014FF000007A
:1007F80070BD41F0FE4141F4780170BD70B54FF015
:10080800FF0C4CF4E06C1CEA11541DBF1CEA135594
:1008180094EA0C0F95EA0C0F00F0A7F8A4EB050476
:1008280081EA030E52EA03354FEA013100F088806D
:100838004FEA03334FF0805545EA131343EA126336
:100848004FEA022245EA111545EA10654FEA0026EB
:100858000EF000419D4208BF964244F1FD0404F5A4
:10086800407402D25B084FEA3202B61A65EB030500
:100878005B084FEA32024FF480104FF4002CB6EBBD
:10088800020E75EB030E22BFB61A754640EA0C003D
:100898005B084FEA3202B6EB020E75EB030E22BF7D
:1008A800B61A754640EA5C005B084FEA3202B6EBBE
:1008B800020E75EB030E22BFB61A754640EA9C007D
:1008C8005B084FEA3202B6EB020E75EB030E22BF4D
:1008D800B61A754640EADC0055EA060E18D04FEA0B
:1008E800051545EA16754FEA06164FEAC30343EAAB
:1008F80052734FEAC2025FEA1C1CC0D111F4801F78
:100908000BD141EA00014FF000004FF0004CB6E770
:1009180011F4801F04BF01430020B4F1FD0C88BF0F
:10092800BCF5E06F3FF6AFAEB5EB030C04BFB6EB1A
:10093800020C5FEA500C50F1000041EB045170BD0D
:100948000EF0004E4EEA113114EB5C04C2BFD4EB3A
:100958000C0541EA045170BD41F480114FF0000EBE
:10096800013C90E645EA060E8DE60CEA135594EA3A
:100978000C0F08BF95EA0C0F3FF43BAF94EA0C0F3D
:100988000AD150EA01347FF434AF95EA0C0F7FF4B2
:1009980025AF104619462CE795EA0C0F06D152EA06
:1009A80003353FF4FDAE1046194622E750EA4106EA
:1009B80018BF52EA43067FF4C5AE50EA41047FF4FB
:1009C8000DAF52EA43057FF4EBAE12E74FF0FF3C60
:1009D80006E000BF4FF0010C02E000BF4FF0010C31
:1009E8004DF804CD4FEA410C7FEA6C5C4FEA430CAA
:1009F80018BF7FEA6C5C1BD001B050EA410C0CBFF9
:100A080052EA430C91EA030F02BF90EA020F00205A
:100A1800704710F1000F91EA030F58BF994208BFC1
:100A280090422CBFD8176FEAE37040F0010070477E
:100A38004FEA410C7FEA6C5C02D150EA013C07D1D5
:100A48004FEA430C7FEA6C5CD6D152EA033CD3D020
:100A58005DF8040B704700BF8446104662468C461A
:100A68001946634600E000BF01B5FFF7B7FF00284D
:100A780048BF10F1000F01BD4DF808EDFFF7F4FF76
:100A88000CBF012000205DF808FB00BF4DF808ED01
:100A9800FFF7EAFF34BF012000205DF808FB00BF24
:100AA8004DF808EDFFF7E0FF94BF012000205DF846
:100AB80008FB00BF4DF808EDFFF7CEFF94BF0120FB
:100AC80000205DF808FB00BF4DF808EDFFF7C4FFF4
:100AD80034BF012000205DF808FB00BF4FEA410247
:100AE80012F5001215D211D56FF47873B3EB625278
:100AF80012D94FEAC12343F0004343EA505311F09F
:100B0800004F23FA02F018BF404270474FF0000030
:100B1800704750EA013005D111F0004008BF6FF06E
:100B2800004070474FF00000704700BF4FEA410295
:100B3800B2F1E04324BFB3F5001CDCF1FE5C0DD933
:100B480001F0004C4FEAC0024CEA5070B2F1004F7D
:100B580040EB830008BF20F00100704711F0804F80
:100B680021D113F13872BCBF01F00040704741F445
:100B780080114FEA5252C2F11802C2F1200C10FA49
:100B88000CF320FA02F018BF40F001004FEAC1232D
:100B98004FEAD32303FA0CFC40EA0C0023FA02F3D1
:100BA8004FEA4303CCE77FEA625307D150EA0133A7
:100BB8001EBF4FF0FE4040F44000704701F0004077
:100BC80040F0FE4040F40000704700BF80F0004055
:100BD80002E000BF81F0004142001FBF5FEA41030D
:100BE80092EA030F7FEA226C7FEA236C6AD04FEA0D
:100BF8001262D2EB1363C1BFD21841404840414052
:100C0800B8BF5B42192B88BF704710F0004F40F403
:100C1800000020F07F4018BF404211F0004F41F41F
:100C2800000121F07F4118BF494292EA030F3FD0EB
:100C3800A2F1010241FA03FC10EB0C00C3F12003FE
:100C480001FA03F100F0004302D5494260EB40008D
:100C5800B0F5000F13D3B0F1807F06D340084FEAF8
:100C6800310102F10102FE2A51D2B1F1004F40EBED
:100C7800C25008BF20F0010040EA03007047490055
:100C880040EB000010F4000FA2F10102EDD1B0FA20
:100C980080FCACF1080CB2EB0C0200FA0CF0AABF15
:100CA80000EBC25052421843BCBFD04018437047B3
:100CB80092F0000F81F4000106BF80F400000132B9
:100CC800013BB5E74FEA41037FEA226C18BF7FEA90
:100CD800236C21D092EA030F04D092F0000F08BFD2
:100CE8000846704790EA010F1CBF0020704712F0B9
:100CF8007F4F04D1400028BF40F00040704712F1F8
:100D080000723CBF00F50000704700F0004343F05C
:100D1800FE4040F4000070477FEA226216BF084692
:100D28007FEA23630146420206BF5FEA412390EA55
:100D3800010F40F4800070474FF0000304E000BF4B
:100D480010F0004348BF40425FEA000C08BF7047FC
:100D580043F0964301464FF000001CE050EA0102C0
:100D680008BF70474FF000030AE000BF50EA0102D5
:100D780008BF704711F0004302D5404261EB4101C2
:100D88005FEA010C02BF84460146002043F0B643E7
:100D980008BFA3F18053A3F50003BCFA8CF2083A0C
:100DA800A3EBC25310DB01FA02FC634400FA02FC15
:100DB800C2F12002BCF1004F20FA02F243EB02001C
:100DC80008BF20F00100704702F1200201FA02FC7E
:100DD800C2F1200250EA4C0021FA02F243EB020071
:100DE80008BF20EADC7070474FF0FF0C1CEAD052B5
:100DF8001EBF1CEAD15392EA0C0F93EA0C0F6FD076
:100E08001A4480EA010C400218BF5FEA41211ED053
:100E18004FF0006343EA501043EA5111A0FB01313F
:100E28000CF00040B1F5000F3EBF490041EAD37114
:100E38005B0040EA010062F17F02FD2A1DD8B3F190
:100E4800004F40EBC25008BF20F00100704790F0FF
:100E5800000F0CF0004C08BF49024CEA502040EA51
:100E680051207F3AC2BFD2F1FF0340EAC250704717
:100E780040F400004FF00003013A5DDC12F1190F55
:100E8800DCBF00F000407047C2F10002410021FAC7
:100E980002F1C2F1200200FA02FC5FEA310040F1DF
:100EA800000053EA4C0308BF20EADC70704792F058
:100EB800000F00F0004C02BF400010F4000F013A90
:100EC800F9D040EA0C0093F0000F01F0004C02BF8B
:100ED800490011F4000F013BF9D041EA0C018FE7FA
:100EE8000CEAD15392EA0C0F18BF93EA0C0F0AD000
:100EF80030F0004C18BF31F0004CD8D180EA010026
:100F080000F00040704790F0000F17BF90F0004FBE
:100F1800084691F0000F91F0004F14D092EA0C0FA0
:100F280001D142020FD193EA0C0F03D14B0218BF33
:100F3800084608D180EA010000F0004040F0FE4079
:100F480040F40000704740F0FE4040F44000704715
:100F58004FF0FF0C1CEAD0521EBF1CEAD15392EA94
:100F68000C0F93EA0C0F69D0A2EB030280EA010C84
:100F780049024FEA402037D04FF0805343EA11111D
:100F880043EA10130CF000408B4238BF5B0042F17B
:100F98007D024FF4000C8B4224BF5B1A40EA0C0020
:100FA800B3EB510F24BFA3EB510340EA5C00B3EB52
:100FB800910F24BFA3EB910340EA9C00B3EBD10F40
:100FC80024BFA3EBD10340EADC001B0118BF5FEA92
:100FD8001C1CE0D1FD2A3FF650AF8B4240EBC250BB
:100FE80008BF20F0010070470CF0004C4CEA50207C
:100FF8007F32C2BFD2F1FF0340EAC250704740F4CB
:1010080000004FF00003013A37E792F0000F00F0BC
:10101800004C02BF400010F4000F013AF9D040EA3A
:101028000C0093F0000F01F0004C02BF490011F4CE
:10103800000F013BF9D041EA0C0195E70CEAD153C6
:1010480092EA0C0F08D142027FF47DAF93EA0C0FAD
:101058007FF470AF084676E793EA0C0F04D14B0291
:101068003FF44CAF08466EE730F0004C18BF31F043
:10107800004CCAD130F000427FF45CAF31F000433D
:101088007FF43CAF5FE700BF4FF0FF3C06E000BFD6
:101098004FF0010C02E000BF4FF0010C4DF804CDF9
:1010A8004FEA40024FEA41037FEA226C18BF7FEA09
:1010B800236C11D001B052EA530C18BF90EA010F0B
:1010C80058BFB2EB030088BFC81738BF6FEAE1709A
:1010D80018BF40F0010070477FEA226C02D15FEA36
:1010E800402C05D17FEA236CE4D15FEA412CE1D0A2
:1010F8005DF8040B704700BF844608466146FFE769
:101108000FB5FFF7C9FF002848BF10F1000F0FBD4A
:101118004DF808EDFFF7F4FF0CBF012000205DF843
:1011280008FB00BF4DF808EDFFF7EAFF34BF0120C8
:1011380000205DF808FB00BF4DF808EDFFF7E0FF61
:1011480094BF012000205DF808FB00BF4DF808EDB2
:10115800FFF7D2FF94BF012000205DF808FB00BF15
:101168004DF808EDFFF7C8FF34BF012000205DF8F7
:1011780008FB00BF4FEA4002B2F1FE4F0FD34FF019
:101188009E03B3EB12620DD94FEA002343F00043EC
:1011980010F0004F23FA02F018BF404270474FF09A
:1011A8000000704712F1610F01D1420205D110F021
:1011B800004008BF6FF0004070474FF000007047D4
:1011C80082B0084B1B68084AA2FB03235B0A00FB9A
:1011D80003F0019000BF019B5A1E0192002BF9D128
:1011E80002B0704700000020D34D621070B582B085
:1011F8000446036813F0010F2CD0AB4B5B6803F077
:101208000C03042B1DD0A84B5B6803F00C03082BC0
:1012180012D06368B3F5803F41D0002B55D103F15C
:10122800804303F504331A6822F480321A601A687E
:1012380022F480221A6037E09B4B5B6813F4803FEE
:10124800E7D0994B1B6813F4003F03D06368002B69
:1012580000F0AE81236813F0020F76D0924B5B68E2
:1012680013F00C0F5FD0904B5B6803F00C03082B56
:1012780054D02369002B00F08A808C4B01221A601D
:1012880000F0F8FF0546884B1B6813F0020F75D174
:1012980000F0F0FF401B0228F5D903208BE1824AB9
:1012A800136843F480331360636843B300F0E2FFCC
:1012B80005467D4B1B6813F4003FCBD100F0DAFFE5
:1012C800401B6428F5D9032075E1B3F5A02F09D098
:1012D800754B1A6822F480321A601A6822F4802248
:1012E8001A60E1E703F18043A3F53C331A6842F43E
:1012F80080221A601A6842F480321A60D4E700F03B
:10130800B9FF0546684B1B6813F4003FA2D000F0F4
:10131800B1FF401B6428F5D903204CE1624B5B68A0
:1013280013F4803FA5D1604B1B6813F0020F04D063
:101338002369012B01D001203DE15B4A136823F0AA
:10134800F803616943EAC1031360236813F0080FC7
:1013580032D0A369002B5BD0554B01221A6000F0F4
:1013680089FF0546504B5B6A13F0020F21D100F04C
:1013780081FF401B0228F5D903201CE14A4A136863
:1013880023F0F803616943EAC1031360DDE7474BC3
:1013980000221A6000F06EFF0546434B1B6813F0ED
:1013A800020FD2D000F066FF401B0228F5D90320B7
:1013B80001E10120FFF704FF236813F0040F00F098
:1013C8009780394BDB6913F0805F33D1364BDA698C
:1013D80042F08052DA61DB6903F080530193019B8C
:1013E8000125344B1B6813F4807F25D0E368012B5B
:1013F80036D0002B4CD103F1804303F504331A6A2D
:1014080022F001021A621A6A22F004021A622CE01F
:10141800274B00221A6000F02DFF0546224B5B6A1D
:1014280013F0020FC8D000F025FF401B0228F5D9A1
:101438000320C0E00025D4E71E4A136843F48073F4
:10144800136000F017FF06461A4B1B6813F4807FE1
:10145800CCD100F00FFF801B6428F5D90320AAE047
:10146800114A136A43F001031362E36873B300F08F
:1014780001FF06460C4B1B6A13F0020F37D100F030
:10148800F9FE801B41F288339842F3D9032092E099
:10149800052B11D0044B1A6A22F001021A621A6A4B
:1014A80022F004021A62E0E7001002400000424203
:1014B8008004424200700040414B1A6A42F0040224
:1014C8001A621A6A42F001021A62CEE700F0D2FEEE
:1014D80006463B4B1B6A13F0020F08D000F0CAFE09
:1014E800801B41F288339842F3D9032063E0E5B9C1
:1014F800E369002B5ED0324A526802F00C02082AD7
:101508005BD0022B17D02F4B00221A6000F0B2FEDE
:1015180004462B4B1B6813F0007F47D000F0AAFE4F
:10152800001B0228F5D9032045E0254AD36923F09A
:101538008053D361DCE7234B00221A6000F09AFE47
:1015480005461F4B1B6813F0007F06D000F092FE83
:10155800401B0228F5D903202DE0236AB3F5803F0C
:101568001AD017494B6823F47413226A606A02433D
:1015780013434B60134B01221A6000F07BFE0446B4
:101588000F4B1B6813F0007F0ED100F073FE001B99
:101598000228F5D903200EE0094A536823F40033E2
:1015A800A1680B435360DCE7002004E0002002E060
:1015B800012000E0002002B070BD0120FBE700BF61
:1015C800001002406000424210B487B0164C94E804
:1015D8000F000DF1180C0CE90F00238AADF8043048
:1015E800124B5B6803F00C02082A1AD1C3F383423A
:1015F800624412F8100C13F4803F05D10C4B03FB26
:1016080000F007B010BC7047084B5B68C3F3404359
:10161800634413F8142C074BB3FBF2F300FB03F0FD
:10162800EFE70448EDE700BF20460008001002403D
:1016380000093D0000127A00594B1B6803F00703AC
:101648008B420CD2564A136823F007030B431360EE
:10165800136803F007038B4201D00120704770B56F
:10166800036813F0020F06D04E4A536823F0F003C4
:101678008468234353600C460546036813F0010F42
:1016880052D04368012B23D0022B28D0454A126838
:1016980012F0020F00F0828042494A6822F00302E9
:1016A80013434B6000F0E6FD06466B68012B1DD026
:1016B800022B2AD03B4B5B6813F00C0F34D000F0A0
:1016C800D9FD801B41F288339842F3D9032064E0A6
:1016D800344A126812F4003FDED101205DE0314A3D
:1016E800126812F0007FD7D1012056E02D4B5B68BD
:1016F80003F00C03042B17D000F0BCFD801B41F253
:1017080088339842F2D9032047E0264B5B6803F000
:101718000C03082B08D000F0ADFD801B41F2883384
:101728009842F2D9032038E01D4B1B6803F00703E9
:10173800A3420CD91A4A136823F007032343136002
:10174800136803F00703A34201D0012025E02B68AA
:1017580013F0040F06D0134A536823F4E063E968D2
:101768000B4353602B6813F0080F07D00D4A5368DA
:1017780023F46053296943EAC1035360FFF724FF48
:10178800084B5B68C3F30313074AD35CD840074B85
:101798001860002000F03EFD002070BD0120FCE72D
:1017A80000200240001002403446000800000020DB
:1017B800014B1868704700BF0000002008B5FFF70C
:1017C800F7FF044B5B68C3F30223034AD35CD8409A
:1017D80008BD00BF001002404446000808B5FFF7E6
:1017E800E7FF044B5B68C3F3C223034AD35CD840CA
:1017F80008BD00BF001002404446000830B4036A28
:1018080023F001030362056A4268846924F07304C3
:101818000B681C4325F002058B682B43104DA8422A
:1018280003D005F50065A84205D123F00803CD686B
:101838002B4323F004030A4DA84203D005F50065A5
:10184800A84205D122F440724D6915438A692A439A
:10185800426084614A684263036230BC704700BFDB
:10186800002C014030B4036A23F480730362036AD6
:101878004268C46924F073040D682C4323F4007390
:101888008D6843EA0523124DA84203D005F500658B
:10189800A84206D123F40063CD6843EA052323F464
:1018A80080630B4DA84203D005F50065A84207D117
:1018B80022F440524D6942EA05128D6942EA051246
:1018C8004260C4614A68C263036230BC704700BFAB
:1018D800002C014030B4036A23F480530362036A86
:1018E8004468C26922F4E6420D6842EA052223F4FC
:1018F80000538D6843EA0533094DA84203D005F526
:101908000065A84204D124F480444D6944EA851452
:101918004460C2614A680264036230BC704700BF19
:10192800002C014010B4036A046A24F00104046224
:10193800846924F0F00444EA021223F00A030B43FA
:101948008261036210BC704710B4036A23F010036D
:1019580003628469036A24F4704444EA023223F07F
:10196800A00343EA01138261036210BC704710B4FC
:10197800846824F47F4442EA03230B4323438360AF
:1019880010BC704710B50468A26822F070024B685A
:10199800134323F007030A681343A3604B68502BD3
:1019A8001ED00AD9602B21D0702B05D10B698A680B
:1019B800C9680068FFF7DBFF10BD402BFCD1036846
:1019C8001C6A1A6A22F001021A620268936923F0FB
:1019D800F003096943EA0113936103681C62EBE7AA
:1019E8000A6989680068FFF79DFFE5E70A69896861
:1019F8000068FFF7A9FFDFE7704738B590F83C307B
:101A0800012B18D00446012580F83C50022380F8A9
:101A18003D30FFF7B7FF2268D36823F04003D36057
:101A28002268D36823F48043D36084F83D500020B3
:101A380084F83C0038BD0220FCE700000368244A13
:101A4800904212D002F5006290420ED0B0F1804F61
:101A58000BD0A2F59832904207D002F580629042EE
:101A680003D002F58062904203D123F070034A68E4
:101A78001343174A904212D002F5006290420ED0EA
:101A8800B0F1804F0BD0A2F59832904207D002F502
:101A98008062904203D002F58062904203D123F421
:101AA8004073CA68134323F080034A6913430360F1
:101AB8008B68C3620B688362054B984203D003F5B9
:101AC8000063984201D10B690363012343617047A6
:101AD800002C0140A8B110B5044690F83D305BB128
:101AE800022384F83D30211D2068FFF7A7FF01235A
:101AF80084F83D30002010BD80F83C30FFF77CFFB3
:101B0800EEE701207047000030B4036A23F01003A9
:101B18000362036A4468826922F4E6420D6842EA75
:101B2800052223F020038D6843EA0513114DA842CE
:101B380003D005F50065A84206D123F08003CD68DF
:101B480043EA051323F040030A4DA84203D005F5E4
:101B58000065A84207D124F440644D6944EA85042D
:101B68008D6944EA8504446082614A68826303623D
:101B780030BC7047002C014038B590F83C30012B40
:101B880066D00D460446012380F83C30022380F8D5
:101B98003D300C2A1AD8DFE802F007191919201964
:101BA80019193419191947000068FFF727FE226828
:101BB800936943F0080393612268936923F004034F
:101BC80093612268936929690B439361012384F81F
:101BD8003D30002084F83C0038BD0068FFF794FFD2
:101BE8002268936943F4006393612268936923F43C
:101BF8008063936122689369296943EA01239361A9
:101C0800E4E70068FFF72EFE2268D36943F0080373
:101C1800D3612268D36923F00403D3612268D369AE
:101C280029690B43D361D1E70068FFF753FE2268A7
:101C3800D36943F40063D3612268D36923F48063D2
:101C4800D3612268D369296943EA0123D361BDE7D7
:101C58000220C1E710B4012303FA01F4036A23EA5E
:101C680004030362036A8A401343036210BC70478B
:101C780010B5044601220068FFF7ECFF2368094A03
:101C8800934203D002F50062934203D15A6C42F4A6
:101C980000425A642268136843F00103136000206D
:101CA80010BD00BF002C014010B4042303FA01F456
:101CB800036A23EA04030362036A8A401343036244
:101CC80010BC704710B5044604220068FFF7ECFF0B
:101CD8002268536C43F4004353642268136843F04A
:101CE80001031360002010BD90F83C30012B25D073
:101CF800012380F83C30CB6823F440738A6813438F
:101D080023F480634A68134323F400630A68134387
:101D180023F480530A69134323F400534A69134395
:101D280023F480438A69134323F40043134302686E
:101D38005364002380F83C301846704702207047EF
:101D480090F83C30012B22D030B4012280F83C209E
:101D5800022380F83D300468636823F070036360F1
:101D6800046863680D682B4363600468A36823F004
:101D78008003A3600468A36849680B43A36080F8E4
:101D88003D20002380F83C30184630BC70470220C4
:101D980070470000034690F82420012A20D0012231
:101DA80080F824200268906810F0010F07D10D48D0
:101DB800806810F0010F02D10B48824208D09A6A5D
:101DC80042F020029A620120002283F82420704702
:101DD800506820F470200968014351600020F3E73F
:101DE800022070470028014000240140074AD368B8
:101DF80023F4E0631B041B0C000200F4E0601843AA
:101E080040F0BF6040F40030D060704700ED00E063
:101E180030B4174BDB68C3F30223C3F10704042C67
:101E280028BF04241D1D062D18D9033B4FF0FF358C
:101E380005FA04F421EA0401994005FA03F322EAB9
:101E48000303194300280BDB0901C9B200F1604004
:101E580000F5614080F8001330BC70470023E5E7C7
:101E680000F00F000901C9B2024B1954F4E700BF92
:101E780000ED00E014ED00E000F01F02400901232E
:101E88009340024A42F82030704700BF00E100E06A
:101E98000138B0F1807F0AD2064B5860064AF0211B
:101EA80082F823100020986007221A6070470120EA
:101EB800704700BF10E000E000ED00E0042805D006
:101EC800054A136823F0040313607047024A136835
:101ED80043F004031360704710E000E0704708B552
:101EE800FFF7FCFF08BD0000F0B482B000263546BD
:101EF800ABE0002C63D0012C00D1CE68FF2B72D848
:101F08008446FF2B72D8AC00DCF800200F27A740CE
:101F180022EA070206FA04F42243CCF800204A68B1
:101F280012F0805F00F09080654A946944F00104E3
:101F38009461926902F001020192019AAC08A71C0F
:101F4800604A52F827C005F0030297000F22BA40F2
:101F58002CEA020C5C4A90424ED002F58062904214
:101F680000F08B8002F58062904200F0888002F5D4
:101F78008062904200F0858002F58062904200F015
:101F8800828002F58062904234D0062235E04F4FBD
:101F9800BC4214D00BD94E4FBC4210D007F5803745
:101FA800BC420CD0A7F58017BC42A7D107E0A7F523
:101FB8008017BC4203D007F58037BC429ED18C689D
:101FC8007CB1012C08D04261082697E7CE68083614
:101FD80094E7CE680C3691E7026108268EE7002662
:101FE8008CE704268AE700F1040C8AE7A5F10804C7
:101FF800A40089E7052200E00022BA4042EA0C0268
:102008000234304F47F824204A6812F4803F3CD00D
:10201800304C22681A4322604A6812F4003F3AD0D2
:102028002C4C62681A4362604A6812F4801F38D0E8
:10203800284CA2681A43A2604A6812F4001F36D0DE
:10204800244CE2681343E36001350F2D35D8012293
:10205800AA400B6813409A42F6D14C68122CB8D0AB
:1020680095D8022CB2D07FF644AF032CB7D0112CF0
:102078007FF444AFCE68043640E70122BDE7022270
:10208800BBE70322B9E70422B7E7124C226822EA29
:1020980003022260C0E70F4C626822EA0302626012
:1020A800C2E70C4CA26822EA0302A260C4E7094C0A
:1020B800E26822EA0303E360C6E702B0F0BC7047B7
:1020C80000100240000001400008014000002110FB
:1020D80000003110000401408368194201D100203A
:1020E80070470120704712B9090401617047016106
:1020F8007047C3685940C1607047000070B582B02E
:102108000446036813F0010F34D03E4BDB6913F02B
:10211800805F48D13B4BDA6942F08052DA61DB6973
:1021280003F080530193019B0125374B1B6813F47F
:10213800807F3AD0334B1B6A13F4407311D0626826
:1021480002F440729A420CD02E4A136A23F440706B
:102158002E4901260E6000260E60106213F0010F52
:1021680037D1284A136A23F4407361680B4313621A
:10217800002D3FD1236813F0020F06D0214A53687F
:1021880023F44043A1680B435360236813F0100FF6
:1021980035D01C4A536823F4800361690B435360AC
:1021A800002002B070BD0025BFE7174A136843F44A
:1021B8008073136000F05EF80646134B1B6813F437
:1021C800807FB7D100F056F8801B6428F5D903202A
:1021D800E7E700F04FF806460A4B1B6A13F0020FB8
:1021E800BFD100F047F8801B41F288339842F3D9F9
:1021F8000320D6E7D36923F08053D361BAE70020E0
:10220800CFE700BF00100240007000404004424287
:102218007047000010B50446074B1868074BA3FB2E
:1022280000308009FFF734FE002221464FF0FF30CE
:10223800FFF7EEFD002010BD00000020D34D621016
:1022480008B5074A136843F0100313600320FFF72B
:10225800CDFD0020FFF7DEFFFFF7DAFF002008BD05
:1022680000200240024A136801331360704700BF20
:10227800E4000020014B1868704700BFE40000200C
:1022880030B583B00190FFF7F5FF0546019CB4F126
:10229800FF3F00D00134FFF7EDFF401BA042FAD307
:1022A80003B030BD7047000030B482B00023019302
:1022B80090F82430012B00F08B800246012380F82F
:1022C80024304B68062B29D80568686B03EB830319
:1022D800053B1F249C4020EA04000C6804FA03F321
:1022E80003436B630B68092B38D91568E86803EB5F
:1022F80043031E3B07249C4020EA04008C6804FA30
:1023080003F30343EB600B68103B012B34D9002027
:10231800002382F8243002B030BC70470C2B0ED852
:102328000568286B03EB8303233B1F249C4020EAAA
:1023380004000C6804FA03F303432B63D2E705682F
:10234800E86A03EB8303413B1F249C4020EA040016
:102358000C6804FA03F30343EB62C3E715682869C2
:1023680003EB430307249C4020EA04008C6804FA2A
:1023780003F303432B61C6E713681648834205D06D
:10238800936A43F0200393620120C1E7986810F430
:10239800000F1BD1986840F4000098600B68102B60
:1023A80001D00020B4E70C4B1B680C49A1FB0313B8
:1023B8009B0C03EB83035900019102E0019B013B55
:1023C8000193019B002BF9D10020A1E700209FE792
:1023D8000220A0E7002401400000002083DE1B4308
:1023E80030B583B00023019303689A6812F0010F97
:1023F8002ED19A6842F001029A60174B1B68174A5F
:10240800A2FB03239B0C019302E0019B013B019378
:10241800019B002BF9D10446FFF72CFF05462368E2
:102428009B6813F0010F11D1FFF724FF401B02280E
:10243800F5D9A36A43F01003A362E36A43F00103EA
:10244800E362002384F82430012002E0002000E049
:10245800002003B030BD00BF0000002083DE1B4316
:1024680090F82430012B6AD010B50446012380F877
:102478002430FFF7B5FF024600285BD1A36A23F496
:10248800407323F0010343F48073A36223682D494A
:102498008B4227D0A16A21F48011A162596811F4F6
:1024A800806F05D0A16A21F4405141F48051A162A6
:1024B800A16A11F4805F2BD0E16A21F00601E16284
:1024C800002184F824106FF00201196023689968CC
:1024D80001F46021B1F5602F1DD0996841F4801195
:1024E80099602AE0A1F58061496811F4702FD1D074
:1024F800A16A41F48011A1621349496811F4806FFF
:10250800D6D0A16A21F4405141F48051A162CFE7AD
:102518000021E162D4E70B498B4204D0996841F469
:10252800A001996009E0A1F58061496811F4702F54
:10253800D3D1F3E7002384F82430104610BD0222DB
:1025480010467047002801400024014038B5036850
:102558009A6812F0010F01D1002038BD04469A682C
:1025680022F001029A60FFF785FE054623689B6802
:1025780013F0010F0ED0FFF77DFE401B0228F5D99E
:10258800A36A43F01003A362E36A43F00103E36222
:102598000120E2E70020E0E7002800F08A8070B51B
:1025A8000446836A002B36D02046FFF7CFFFA36A84
:1025B80013F0100377D1002875D1A26A22F488524B
:1025C80022F0020242F00202A262626825683A49D9
:1025D8008D4226D0E1690A43E66842EA4602A168CC
:1025E800B1F5807F27D0012922D06169012925D042
:1025F800696821F469410B436B6021688D682F4B32
:102608002B4013438B60A368B3F5807F27D0012B41
:1026180025D0002126E0C36280F82430FFF742FE6F
:10262800C2E7E169B1F5402FD5D14FF40021D2E7D7
:102638004FF48073D9E74FF48073D6E736B9A169B0
:10264800013943EA413343F40063D1E7A16A41F019
:102658002001A162E16A41F00101E162C8E7236952
:10266800013B19052568EB6A23F470030B43EB6201
:1026780023689968124B0B409A420BD0A36A23F047
:10268800120343F01003A362E36A43F00103E36219
:1026980001200DE00023E362A36A23F0030343F063
:1026A8000103A36204E0A36A43F01003A3620120BC
:1026B80070BD0120704700BF003C0140FDF7E1FFFD
:1026C800FE0E1FFF2DE9F84305460268136923F43F
:1026D8004053C1680B43136183680269134342691D
:1026E80013430168CA6822F4B05222F00C02134363
:1026F800CB600268536923F4407381690B435361CB
:102708000268594B9A4257D0FFF758F800EB8000FF
:1027180000EB80006C68A400B0FBF4F4534FA7FBF7
:10272800043464092601FFF749F800EB800000EB48
:1027380080006C68A400B0FBF4F9FFF73FF800EBE9
:10274800800000EB80006C68A400B0FBF4F4A7FBE9
:10275800043464094FF0640808FB149424013234EB
:10276800A7FB0434640904F0F0043444FFF726F8A6
:1027780000EB800000EB80006E68B600B0FBF6F658
:10278800FFF71CF800EB800000EB80006B689B00F3
:10279800B0FBF3F0A7FB0030400908FB10684FEAD4
:1027A800081808F13208A7FB0837C7F343172B6846
:1027B80027449F60BDE8F883FFF710F800EB80001E
:1027C80000EB80006C68A400B0FBF4F4274FA7FB73
:1027D800043464092601FFF701F800EB800000EBE0
:1027E80080006C68A400B0FBF4F9FEF7F7FF00EB7B
:1027F800800000EB80006C68A400B0FBF4F4A7FB39
:10280800043464094FF0640808FB1494240132343A
:10281800A7FB0434640904F0F0043444FEF7DEFF37
:1028280000EB800000EB80006E68B600B0FBF6F6A7
:10283800FEF7D4FF00EB800000EB80006B689B0084
:10284800B0FBF3F0A7FB0030400908FB10684FEA23
:10285800081808F13208A7FB0837C7F343172B6895
:1028680027449F60A6E700BF003801401F85EB5151
:10287800704758B310B5044690F839300BB3242389
:1028880084F839302268D36823F40053D360204693
:10289800FFF718FF2268136923F490431361226835
:1028A800536923F02A0353612268D36843F4005321
:1028B800D3600020E063202384F8393084F83A306C
:1028C80010BD80F83830FFF7D3FFD8E701207047F4
:1028D8000F4B1A6842F001021A6059680D4A0A4003
:1028E8005A601A6822F0847222F480321A601A68D8
:1028F80022F480221A605A6822F4FE025A604FF4C9
:102908001F029A60044B4FF000629A60704700BF44
:10291800001002400000FFF800ED00E030B597B06D
:102928001F4BDA6942F48022DA61DA6902F4802204
:102938000092009A5A6942F001025A615B6903F0F9
:1029480001030193019B174D06954FF4E13307935B
:102958000024089409940A9408230B930C940D946A
:1029680006A8FFF786FF6B6943F080036B614FF49D
:1029780080630293012304930223039303230593A3
:1029880002A90948FFF7B0FA084B1C60084A9A6088
:102998005C6090221A601C3B70225A6017B030BDF0
:1029A8000010024000480040000C01401C0002409A
:1029B800044800402DE9F04F89B07B4B9A6942F0FA
:1029C80004029A619A6902F004020192019A9A69D2
:1029D80042F008029A619A6902F008020292029A89
:1029E8009A6942F010029A619B6903F010030393FD
:1029F800039B002305930693022707974FF0200AAD
:102A08000DEB0A0444F810AD21466848FFF76CFA4C
:102A18004023049321466548FFF766FA802504950C
:102A280021466248FFF760FA4FF480630493214619
:102A38005F48FFF759FA4FF40063049321465C4856
:102A4800FFF752FA4FF48056049621465848FFF78C
:102A58004BFA049621465748FFF746FA0497214651
:102A68005448FFF741FA4FF00108CDF814804FF0B1
:102A78000409CDF8109021464C48FFF735FA102686
:102A8800049621464B48FFF72FFACDF810A02146AF
:102A98004848FFF729FA03230593CDF8108021460B
:102AA8004348FFF721FACDF8108021464148FFF747
:102AB8001BFA4FF0080BCDF810B021463C48FFF741
:102AC80013FA049721463A48FFF70EFA049621466E
:102AD8003748FFF709FACDF810A021463448FFF728
:102AE80003FACDF8109021463148FFF7FDF9CDF8EB
:102AF80010B021462F48FFF7F7F9CDF8109021467E
:102B08002C48FFF7F1F905974023049321462848FC
:102B1800FFF7EAF9049521462548FFF7E5F94FF450
:102B28008079CDF8109021462148FFF7DDF904950A
:102B380021462048FFF7D8F9CDF8108021461B48D8
:102B4800FFF7D2F9049721461848FFF7CDF9CDF8D9
:102B5800109021461748FFF7C7F94FF40073049304
:102B680021461448FFF7C0F94FF4806304932146C7
:102B78001048FFF7B9F94FF40053049321460B4866
:102B8800FFF7B2F94FF48043049321460748FFF753
:102B9800ABF94FF40043049321460448FFF7A4F926
:102BA80009B0BDE8F08F00BF00100240000C0140E2
:102BB80000100140000801402DE9F04F99B0754B15
:102BC8009A6942F400629A619A6902F40062019279
:102BD800019A9A6942F400529A619B6903F400537E
:102BE8000293029B6C4EDFF8B891C6F8009000245F
:102BF80074604FF02008C6F808804FF4FA6BC6F8E6
:102C08000CB034617461B4613046FEF763FF102381
:102C18001693179416A93046FFF792F860230F937E
:102C28001094119408271297139414944FF4007376
:102C3800159322460FA93046FEF79EFF04220FA9DE
:102C48003046FEF799FF3A460FA93046FEF794FF43
:102C58004FF4006308934FF4806309930A94CDF806
:102C68002C800C940D940E940DEB08013046FFF760
:102C78003BF84A4DDFF82CA1C5F800A06C60C5F8F8
:102C88000880C5F80CB02C616C61AC612846FEF771
:102C980021FFCDF858808023179316A92846FFF7FF
:102CA8004FF8049418A9052341F8543D2846FEF727
:102CB800A4FE60230F931094119412971394149404
:102CC8004FF40073159322460FA92846FEF754FFC8
:102CD80004220FA92846FEF74FFF3A460FA92846B7
:102CE800FEF74AFF4FF4006308934FF4806309939B
:102CF8000A94CDF82C800C940D940E940DEB0801D9
:102D08002846FEF7F1FFDAF8443023F40043CAF806
:102D18004430D9F8443023F40043C9F844302146FC
:102D28002846FEF7A5FF04212846FEF7A1FF3946ED
:102D38002846FEF79DFF21462846FEF7C3FF0421DB
:102D48002846FEF7BFFF39462846FEF7BBFF214657
:102D58003046FEF78DFF04213046FEF789FF3946DD
:102D68003046FEF785FF21463046FEF7ABFF0421CB
:102D78003046FEF7A7FF39463046FEF7A3FF2B681B
:102D880001221A633268136843F00103136019B013
:102D9800BDE8F08F00100240B00100204003002081
:102DA800002C0140003401402DE9F04186B0424E2C
:102DB800B36943F40073B361B36903F40073009318
:102DC800009B3E4C3E4B23604FF48073A36000256C
:102DD800E56065614FF44023E36165604FF00508E5
:102DE800C4F810802046FFF7D7FB364A536843F4EF
:102DF8008023536006A94FF4C02341F8043D2046C0
:102E0800FEF7C8FF012304930E220292039302A93E
:102E18002046FFF749FA02950227039702A92046A0
:102E2800FFF742FA04970B2702970323039302A99B
:102E38002046FFF739FA0C2302930423039302A9CF
:102E48002046FFF731FA0723049310230293CDF8A5
:102E58000C8002A92046FFF727FA2268936843F4FA
:102E6800000343F480739360936843F00103936015
:102E7800736943F001037361736903F001030193FC
:102E8800019B114B1D60C3F80480104A9A60104AD8
:102E9800DA6040F6A2221A601A6842F001021A604B
:102EA8002A4629463846FEF7B3FF3846FEF7E4FFC0
:102EB80006B0BDE8F08100BF001002407802002093
:102EC8000024014000000140080002404C24014059
:102ED800EC020020F0B585B0284B9A6942F4806274
:102EE8009A619B6903F480630093009B244C254BF3
:102EF80023604FF48073A3600023E36063614FF4A1
:102F08006022E2616360052626612046FFF744FBE4
:102F1800012303930F220192029301A92046FFF790
:102F2800C3F90D2301930225029501A92046FFF755
:102F3800BBF903950A2301930327029701A92046A9
:102F4800FFF7B2F90195042302930DEB0301204624
:102F5800FFF7AAF9072303930197029601A92046D0
:102F6800FFF7A2F923689A6842F480729A609A6817
:102F780042F001029A6005B0F0BD00BF00100240A7
:102F88002C0100200028014010B50024094B1C70BA
:102F9800094B1C7005E0094B1C706420FFF770F9A1
:102FA8000134072CF7DD002220210548FFF79BF8A4
:102FB800FEE700BFAC000020B8000020A8000020F9
:102FC8000008014030B597B002250C9501231093F5
:102FD800102311931395002414944FF46013159340
:102FE8000CA8FEF703F90F230793089509944FF4EB
:102FF80080630A930B94294607A8FEF71DFB0195E9
:103008004FF44043039301A8FFF778F8FEF7D0FB8D
:10301800084BA3FB00308009FEF73AFF0420FEF7B7
:103028004DFF224621464FF0FF30FEF7F1FE17B064
:1030380030BD00BFD34D62102DE9F04F85B0FFF7CA
:10304800FFF8AB4CA36943F00103A361A36903F044
:1030580001030393039B0320FEF7C8FE00221146D9
:103068006FF00B00FEF7D4FE002211466FF00A0045
:10307800FEF7CEFE002211466FF00900FEF7C8FEEB
:10308800002211466FF00400FEF7C2FE002211462E
:103098006FF00300FEF7BCFE002211466FF001003E
:1030A800FEF7B6FE002211464FF0FF30FEF7B0FEE5
:1030B800FFF788FF636923F001036361FFF77AFC78
:1030C800FFF77AFDFFF770FEFFF704FFFFF726FC16
:1030D800012220218748FFF706F88748FFF7C0F943
:1030E8008648FFF7BDF9082405E0854B1C7064206D
:1030F800FFF7C6F8013C002CF7DA4FF0000A804BC6
:1031080083F800A0012204217E48FEF7ECFF7E4BE5
:10311800188AFDF711FE01907C4B01221A70D346E4
:1031280044E17B490A6801320A604BE14FF47A783E
:1031380032463B4620462946FDF780F804460D46B0
:103148000022744BFDF7C0FC88B963A3D3E90023C0
:1031580020462946FDF79AFC00285DD120462946DD
:10316800FDF7BCFC044604E0DFF8DC81E0E74FF43F
:103178007A740AF13203A34215DDAAF1320AA24594
:1031880011DA0BF1320343450DDDABF1320BC345C8
:1031980009DA614B1B68042B05D8604BC3F8008023
:1031A80063425F4A13605F4B1A685F4BA3FB0213CD
:1031B800DB0803EB830303EB83039A422ED002213F
:1031C8004C48FEF789FF30B1584B1B681BB9584B68
:1031D8001B68002B73D0574B1D6857492846FDF7CD
:1031E800A1FF20B1554B1B681333262B72D95449C4
:1031F8002846FDF797FF002800F0B0804E49284682
:10320800FDF7AEFF002800F0A9803D4B05221A709B
:103218004C4B06221A70ADE04B4CAAE70198FDF71B
:103228006BF92FA3D3E90023FDF7BEF906460F4635
:10323800354D288AFDF780FDFDF75EF92AA3D3E90D
:103248000023FDF7B1F902460B4630463946FCF734
:10325800F5FFFDF76BFC074601903C49FDF7BAFC0A
:103268003B49FDF7C1FD3B49FDF7B6FC0646414623
:10327800022000F001FD2146032000F0FDFCA98991
:10328800042000F0F9FC34492A4B1868FDF7ACFD1E
:10329800FDF770FF0146052000F0EEFC3846FDF70B
:1032A80069FF0146062000F0E7FC3046FDF762FFA3
:1032B8000146072000F0E0FC00F0E4FC7FE7134B38
:1032C80000221A7002210B48FEF706FF0028F9D1E8
:1032D800FFF75AFEFFF758FE0000000000408FC0BD
:1032E800AE47E17A14AEEF3F7B14AE47E17A843FF4
:1032F8000010024000080140780200202C01002044
:10330800A8000020000C0140EC020020B8000020BA
:103318009003002000408F4004000020CC000020D3
:10332800C8000020800300201F85EB51D400002036
:10333800D00000200C0000208FC221429C030020F6
:1033480000002842AC00002018FCFFFF00E0CE443B
:10335800083748BE33330F420000C842664B1B682B
:1033680013F1320F80F2AD80644B05221A70644B62
:1033780001221A7084EAE473A3EBE473322B06DCAF
:1033880088EAE873A3EBE873322B40F3A0805D4B27
:1033980000221A605B4B1A685B4B9A4200F29C80D1
:1033A8005A4A136801331360A246C3460520FEF744
:1033B80067FF574B1B68012B3FF4B3AE55490A68AA
:1033C800013A0A60534A176887EAE772A2EBE77284
:1033D800B2F5967F02DD5B424D4A13604E4B0022E8
:1033E8001A60DFF84481D8F80000FDF773F83CA3B1
:1033F800D3E90023FDF7D8F804460D46474B186873
:10340800FDF768F838A3D3E90023FDF7CDF80246A5
:103418000B4620462946FCF711FFFDF75FFB0646E1
:10342800C8F80000DFF8D080D8F80000FDF752F89F
:103438002BA3D3E90023FDF7B7F804460D46384619
:10344800FDF748F828A3D3E90023FDF7ADF80246B5
:103458000B4620462946FCF7F1FEFDF73FFBC8F86E
:103468000000FDF737F800222D4BFDF79DF80446C4
:103478000D463046FDF72EF80022294BFDF794F84B
:1034880006460F4602460B4620462946FCF7D4FE60
:10349800804689460022234BFDF716FB00287FF45F
:1034A80045AE13A3D3E9002340464946FDF7EEFA9B
:1034B80000287FF459AE40464946FDF70FFB804689
:1034C80036E600230D4A13700D4A137052E70D4A71
:1034D8001368013313605DE7FFF756FDAFF3008013
:1034E800666666666666EE3F9A9999999999A93FC4
:1034F8000000000000408FC09C030020A8000020AE
:10350800AC000020840300208038010080030020E4
:10351800080000209003002004000020A4030020DD
:103528000000E03F00408F409403002000000000AE
:10353800774B02225A60774B1B68B3F57A7F5EDBC4
:103548002DE9F041744B1A68744BA3FB02139B09D5
:103558004FF47A7101FB13230BBB714C2068FCF705
:10356800CBFF65A3D3E90023FDF71EF806460F46F7
:103578006C4B9889FDF7E0FB6B49FDF735FCFCF7D0
:10358800BBFF5FA3D3E90023FDF70EF802460B4605
:1035980030463946FCF752FEFDF7C8FA2060614B09
:1035A8005889624B1C68001BFCF794FF56A3D3E9AB
:1035B8000023FCF7F9FF00220023FDF767FA002833
:1035C80052D1584B5889001BFCF784FF4EA3D3E90E
:1035D8000023FCF7E9FF0022554BFDF775FA002898
:1035E80052D1544B1B68052B4ED8534B1B78002BDC
:1035F8004AD0524A536C43F40043536449E00133C0
:10360800444A1360474A90884D490B68034403EBCA
:10361800D3735B100B60D0884A490B68034403EBF3
:10362800D3735B100B60108847490B68034403EBA6
:10363800D3735B100B60508844490B68034403EB59
:10364800D3735B100B60508938490B68034403EB54
:10365800D3735B100B6011893D4A13680B4403EB6D
:10366800D3735B10136070472E4B5889001BFCF70F
:1036780031FF25A3D3E90023FCF796FF0022354B41
:10368800FDF704FA0028ACD02C4A536C23F400430D
:103698005364244B18892E4B1C68001BFCF71AFF37
:1036A80019A3D3E90023FCF77FFF00220023FDF7CD
:1036B800EDF9002852D11B4B1889001BFCF70AFFB3
:1036C80011A3D3E90023FCF76FFF0022184BFDF785
:1036D800FBF9002852D1174B1B68052B4ED8164B07
:1036E8001B78002B4AD01C4A536C43F400435364A4
:1036F80049E000BFAFF30080AE47E17A14AEEF3F78
:103708007B14AE47E17A843F7B14AE47E17A943F5D
:1037180000000240BC000020B0000020D34D621021
:103728000C000020EC02002017B9CE3C100000204D
:1037380000002E4004000020B800002000340140A2
:10374800180000201C000020200000202400002079
:103758001400002000002EC0002C0140904B188956
:10376800001BFCF7B7FE8CA3D3E90023FCF71CFF72
:1037780000228C4BFDF78AF90028ACD08A4A536C9A
:1037880023F40043536489498B6813F0200F0CBF5E
:10379800012300238A6812F0400F0CBF0122002287
:1037A800896811F0800F0CBF0125002580498868C1
:1037B80010F4806F0CBF012000208C6814F4006F97
:1037C8000CBF01240024896811F4805F02EB4502D4
:1037D80003EB4203774EF35C77490B600B6803F108
:1037E80002030B600D68754B83FB0572A2EBE57253
:1037F80002EB42024FEA4207A5EB07020A600CBF40
:1038080002220022224400EB4202B05C6C4A1060A3
:10381800106802301060106883FB0043A3EBE0736C
:1038280003EB43035C00031B136009685C4883884F
:10383800644A12689A1AC388634800681B1A0529E3
:1038480034D8DFE801F0032326292C2FD31A5F4A46
:1038580013605F4A1368013313605E4A14684CB3FF
:103868005D4AA2FB0312120B5C4909680131B2FBE5
:10387800F1F001FB1022EAB9B3FBF4F204FB1233B6
:10388800EBB910215648FEF734FC18E04F4B1A608C
:10389800DFE74E4B1A60DCE74C4A1360D9E74B4A26
:1038A8001360D6E79B1A494A1360D2E7474B0022B8
:1038B8001A60CEE7002210214948FEF714FC494B54
:1038C800D3F800C03C4B1B68052B2BD8DFE803F06E
:1038D8000312171C2226CCF1000064469C46424B7A
:1038E8001968374B1B68052B52D8DFE803F01F3FD8
:1038F80043474B4E6446CCF1000C0020EFE760468E
:10390800CCF1000C0024EAE7CCF1000460464FF04B
:10391800000CE4E7CCF100040020E0E7CCF1000063
:103928000024DCE7002004468446D8E74E420F46D0
:1039380019462C4B1B68002B40F398802B4B1D68B5
:103948001D4B1B6805331D4A82FB03E2A2EBE372A1
:1039580002EB42024FEA420EA3EB0E02052A00F2E6
:10396800B980DFE802F0456A6F74797E0F464942F4
:103978000026DEE70E4649420027DAE74F420E46A8
:103988000021D6E74F420026D3E74E420027D0E772
:10399800002637463146CCE77B14AE47E17A943FA0
:1039A800EC02002000002EC0002C0140000C014059
:1039B800001001404C460008C0000020ABAAAA2A0B
:1039C800C4000020180000201C000020B4000020C3
:1039D800B0000020A80000205917B7D1AC00002083
:1039E80000080140C8000020CC000020D0000020C2
:1039F800C5F10008AE461546654474444044964BEC
:103A08001B68002B40F3D780944B1B68944A1268BC
:103A180002F1050C934A82FB0CE2A2EBEC7202EB7A
:103A280042024FEA420EACEB0E02052A00F2F98080
:103A3800DFE802F058A8ADB2B7BCAE466D424FF011
:103A48000008D9E7A8466D424FF0000ED4E7C5F14B
:103A5800000EA8460025CFE7C5F1000E4FF000087C
:103A6800CAE7C5F100084FF0000EC5E77E4B1D6898
:103A7800C5F1000E7D4B1A6801327A4B83FB028335
:103A8800A3EBE27303EB43034FEA4308A2EB0803FB
:103A9800052B1AD8DFE803F00323060A0E14A846FC
:103AA8001D46A9E7F0464FF0000EA5E7F046AE46E2
:103AB8000025A1E72B4675469E464FF000089BE778
:103AC800A84675464FF0000E96E74FF00008C64628
:103AD800454691E74FF00008C64645468CE74FF04B
:103AE800000889E7C3F100089E461346194407EB0E
:103AF8000E0206EB080305F57A7540F2C676B54264
:103B080000F397800A2DB8BF0A25594E756304F54E
:103B18007A7440F2C675AC4200F38E800A2CB8BFA6
:103B28000A24534DAC6300F57A7040F2C674A04283
:103B380000F385800A28B8BF0A204D4CE06301F5E0
:103B48007A7140F2C67081427CDC0A29B8BF0A212A
:103B58004848416302F57A7240F2C6718A4274DCC1
:103B68000A2AB8BF0A2243498A6303F57A7340F2E6
:103B7800C67293426CDC0A2BB8BF0A233D4AD36352
:103B8800BDE8F0819E465B424FF00008AEE79846DC
:103B98005B424FF0000EA9E7C3F1000E98460023E0
:103BA800A4E7C3F1000E4FF000089FE7C3F1000837
:103BB8004FF0000E9AE7294B1B68C3F1000E284A04
:103BC80012680132DFF89CC08CFB028CACEBE27C03
:103BD8000CEB4C0C4FEA4C08A2EB080CBCF1050F9F
:103BE8001AD8DFE80CF00323060A0E149846634639
:103BF8007CE7F0464FF0000E78E7F0469E4600233B
:103C080074E71A46734696464FF000086EE79846E2
:103C180073464FF0000E69E74FF00008C64643466A
:103C280064E74FF00008C64643465FE74FF00008D8
:103C38005CE740F2C67568E740F2C67471E740F287
:103C4800C6707AE740F2C67182E740F2C6728AE728
:103C580040F2C67392E700BFCC000020D4000020D9
:103C6800C4000020ABAAAA2AD0000020C00000206F
:103C780000340140002C0140014B23F8101070471C
:103C88000C040020F0B587B01A4F64220021384692
:103C980000F090F818490A88B1F802C0888800B284
:103CA800CC8824B20D892DB24E8936B28B891BB2CD
:103CB800C98909B20591049303960295019400906D
:103CC8000FFA8CF312B20D49384600F07BF80C4B12
:103CD8005B686BB90A4C236823F0010323603846FC
:103CE800FCF79EFA6060E760236843F001032360F5
:103CF80007B0F0BDA80300200C04002054460008BB
:103D08001C0002407047FEE7FEE7FEE7FEE770474B
:103D18007047704708B5FEF7A5FAFEF7E0F808BD4A
:103D2800002103E00B4B5B58435004310A480B4B0E
:103D380042189A42F6D30A4A02E0002342F8043BAA
:103D4800084B9A42F9D3FEF7C3FD00F00FF8FFF7CE
:103D580073F97047BC460008000000208C00002062
:103D68008C00002020040020FEE7000070B500252C
:103D78000C4E0D4CA41BA410A54209D100F040FC28
:103D880000250A4E0A4CA41BA410A54205D170BDFB
:103D980056F8253098470135EEE756F8253098470C
:103DA8000135F2E7B4460008B4460008B4460008F6
:103DB800B846000803460244934200D1704703F80E
:103DC800011BF9E70EB46FF0004100B59CB01DABC4
:103DD80002900690079104910848094953F8042B6A
:103DE8000591006802A9019300F066F80022029B81
:103DF8001A701CB05DF804EB03B07047280000206F
:103E08000802FFFF2DE9F0478E6882469E420C4665
:103E18009046994637D88A8912F4906F31D0022398
:103E2800256809696F1A656905EB450595FBF3F582
:103E380009F101033B449D4238BF1D46530530D567
:103E4800294600F035FB064650B90C234FF0FF30E9
:103E5800CAF80030A38943F04003A381BDE8F08786
:103E68003A46216900F0B4FAA38923F4906343F039
:103E78008003A38126613E4426604E466561ED1BA2
:103E8800A5604E4500D94E4632464146206800F0AE
:103E9800AAFAA36800209B1BA36023681E4426601F
:103EA800DCE72A4600F05EFB06460028E2D12169DD
:103EB800504600F0B1FAC8E72DE9F04F9DB00393E2
:103EC8008B8980461D060C4616460FD50B696BB9C3
:103ED800402100F0EDFA2060206128B90C23C8F8D1
:103EE80000304FF0FF30C7E040236361002309939F
:103EF80020238DF8293030234FF0010B8DF82A301C
:103F080037463D4615F8013B0BB1252B3ED1B7EBA3
:103F1800060A0BD05346324621464046FFF772FF49
:103F2800013000F0A480099B534409933B78002B8F
:103F380000F09D8000234FF0FF32CDE90523049364
:103F480007938DF853301A932F46052217F8011B53
:103F58004F4800F02FFA049BD0B9D90644BF20225D
:103F68008DF853201A0744BF2B228DF853202A7846
:103F78002A2A15D02F4600200A25079A394611F813
:103F8800013B303B092B4DD9B8B10FE02F46B8E7BC
:103F98003F4A3D46801A0BFA00F018430490D3E7D5
:103FA800039A111D12680391002A01DB079204E0AD
:103FB800524243F00203079204933B782E2B0CD114
:103FC8007B782A2B33D1039B02371A1D1B68039277
:103FD800002BB8BF4FF0FF3305932E4D03223978DD
:103FE800284600F0E7F938B14023401B03FA00F0F7
:103FF800049B0137034304933978062226487E1C24
:104008008DF8281000F0D6F9002838D0234B13BBC0
:10401800039B073323F0070308330393099B4B449F
:1040280009936DE705FB023201200F46A6E700233E
:104038000A25194601370593384610F8012B303AFE
:10404800092A03D9002BC8D00591C6E705FB012131
:1040580001230746F0E703AB00932246104B04A95F
:104068004046AFF30080B0F1FF3F8146D6D1A38927
:104078005B063FF536AF09981DB0BDE8F08F03AB7E
:1040880000932246064B04A9404600F081F8EAE76F
:1040980080460008864600088A460008000000009E
:1040A8000D3E00082DE9F04791461F468A680B69C6
:1040B80006469342B8BF1346C9F8003091F843202A
:1040C8000C46DDF8208012B10133C9F800302368AE
:1040D800990642BFD9F800300233C9F80030256884
:1040E80015F0060507D104F1190AE368D9F800208C
:1040F8009B1AAB4229DC94F843302268003318BF7E
:10410800012392062ED404F1430239463046C047B3
:10411800013021D02368E56803F00603042B18BF9B
:104128000025D9F800204FF0000908BFAD1AA36890
:10413800226908BF25EAE5759342C4BF9B1AED18AA
:104148001A344D451AD1002008E001235246394659
:104158003046C047013003D14FF0FF30BDE8F0874B
:104168000135C2E73020E11881F843005A1C94F861
:1041780045102244023382F84310C4E70123224643
:1041880039463046C0470130E6D009F10109D8E781
:104198002DE9F04301F1430C0C46097E85B06E29E8
:1041A8001746064698460C9A00F0B38022D8632931
:1041B80036D00AD8002900F0B980582900F0838049
:1041C80004F1420584F8421032E0642901D06929DB
:1041D800F6D120681368050603F104012AD51B6887
:1041E8001160002B03DA2D225B4284F843206F48CC
:1041F8000A2239E0732900F09D8008D86F2920D061
:104208007029DDD1236843F02003236003E075297A
:1042180017D07829D4D17823654884F8453055E0FB
:10422800136804F14205191D1B68116084F84230B7
:1042380001238CE01B6810F0400F116018BF1BB2FF
:10424800CFE713682568181D1060280601D51B687C
:1042580002E06806FBD51B886F2914BF0A220822D2
:104268005248002184F843106568002DA560C0F20B
:104278009580216821F004012160002B3DD1002D9B
:1042880040F08E806546082A0BD12368DB0708D5E5
:10429800236962689A42DEBF302305F8013C05F1C4
:1042A800FF35ACEB05032361CDF800803B4603AA3C
:1042B80021463046FFF7F6FE01304DD14FF0FF3072
:1042C80005B0BDE8F083394884F8451013682168C3
:1042D8001D1D1B6815600A060BD5CA0744BF41F0AF
:1042E800200121601BB9226822F0200222601022DE
:1042F800B7E74D0648BF9BB2EFE76546B3FBF2F15F
:1043080002FB1133C35C05F8013D0B460029F5D1CA
:10431800B9E713682568181D6169106028061B68CD
:1043280001D5196002E06A06FBD5198000236546AD
:104338002361B9E71368191D11601D6862680021BF
:10434800284600F037F808B1401B606063682361B5
:10435800002384F84330A7E723692A4639463046C4
:10436800C0470130AAD023689B0713D4E068039B99
:104378009842B8BF1846A3E701234A463946304653
:10438800C04701309AD00135E368039A9B1AAB42C3
:10439800F2DCEBE7002504F11909F5E7002BACD1B5
:1043A800037804F1420584F842306CE7914600082E
:1043B800A246000810B5C9B202449042034601D192
:1043C800002303E01C7801308C42F6D1184610BD5A
:1043D80010B5431E0A44914200D110BD11F8014B9B
:1043E80003F8014FF7E7884210B501EB020307D83D
:1043F800421E99420AD011F8014B02F8014FF8E722
:104408008342F5D98118D21AD34200D110BD13F8CE
:10441800014D01F8014DF7E738B50546002943D0AD
:1044280051F8043C0C1F002BB8BFE41800F0D0F87A
:104438001E4A1368104633B9636014602846BDE805
:10444800384000F0C6B8A3420BD9216862189342DD
:1044580001BF1A685B685218226063600460EDE768
:1044680013465A680AB1A242FAD919685818A042E4
:104478000BD120680144581882421960DED11068B7
:104488005268014419605A60D8E702D90C232B609E
:10449800D4E7206821188A4201BF116852680918B8
:1044A800216062605C60C9E738BD00BFD8000020A9
:1044B80070B5CD1C25F0030508350C2D38BF0C252B
:1044C800002D064601DBA94203D90C2333600020E6
:1044D80070BD00F07DF8214A1468214691B9204C3E
:1044E80023681BB9304600F063F82060294630463F
:1044F80000F05EF8431C24D10C233046336000F0F2
:1045080068F8E4E70B685B1B18D40B2B0FD90B601A
:10451800CC18CD50304600F05CF804F10B00231D98
:1045280020F00700C31AD3D05A42E250D0E74B68B4
:104538008C4216BF636013600C46EBE70C46496873
:10454800CCE7C41C24F00304A04205D0211A30464D
:1045580000F02EF80130CFD02560DBE7D80000202E
:10456800DC000020F8B5074614460E4621B9BDE820
:10457800F8401146FFF79CBF22B9FFF74DFF2546CB
:104588002846F8BD00F026F8A0420FD2214638464A
:10459800FFF78EFF05460028F2D031462246FFF786
:1045A80017FF31463846FFF737FFE9E73546E7E7B3
:1045B80038B50023054C05460846236000F012F87C
:1045C800431C02D1236803B12B6038BD1C040020B2
:1045D8007047704751F8043C181F002BBCBF0B589C
:1045E800C0187047044A05491368002B08BF0B46DA
:1045F8001844106018467047E0000020200400208E
:10460800F8B500BFF8BC08BC9E467047F8B500BFB7
:08461800F8BC08BC9E46704787
:1046200002030405060708090A0B0C0D0E0F1010F3
:10463000010200000000000000000000010203046D
:10464000060708090000000001020304000002013F
:1046500004050300313A256920323A256920333AAE
:10466000256920343A256920353A256920363A25CE
:104670006920373A256920383A25690D0A0000007B
:10468000232D302B2000686C4C006566674546473B
:1046900000303132333435363738394142434445BE
:1046A000460030313233343536373839616263642D
:0446B000656600003B
:0446B4000D020008EB
:0446B800E90100080C
:1046BC0000A24A0464000000010000000000404217
:1046CC00D0070000D0070000D0070000D007000082
:1046DC00D0070000D00700002C00002000000000D4
:1046EC0000000000000000000000000000000000BE
:1046FC0000000000000000000000000000000000AE
:10470C00000000000000000000000000000000009D
:10471C00000000000000000000000000000000008D
:10472C00000000000000000000000000000000007D
:0C473C0000000000000000000000000071
:0400000508003D2989
:00000001FF
